LINK : warning L4021: no stack segment

 Start  Stop   Length Name                   Class
 00000H 00000H 00000H DNLTCLNT_TEXT          CODE
 00000H 001BDH 001BEH EXPORTLT_TEXT          CODE
 001BEH 002ABH 000EEH DNETADDR_TEXT          CODE
 002ACH 003ADH 00102H DNETPATH_TEXT          CODE
 003AEH 0040FH 00062H GNODEBAD_TEXT          CODE
 00410H 0048DH 0007EH GNODEBNM_TEXT          CODE
 0048EH 005BFH 00132H GNODEENT_TEXT          CODE
 005C0H 005F3H 00034H HCLOSE_TEXT            CODE
 005F4H 00691H 0009EH HOPEN_TEXT             CODE
 00692H 006F5H 00064H HREAD_TEXT             CODE
 006F6H 0078DH 00098H HSEEK_TEXT             CODE
 0078EH 007EDH 00060H PRGCLS_TEXT            CODE
 007EEH 00841H 00054H PRGCON_TEXT            CODE
 00842H 00953H 00112H PRGRCV_TEXT            CODE
 00954H 00A3FH 000ECH PRGSEL_TEXT            CODE
 00A40H 00B3BH 000FCH PRGSND_TEXT            CODE
 00B3CH 00B95H 0005AH PRGSOC_TEXT            CODE
 00B96H 00BB3H 0001EH PTRCONV_TEXT           CODE
 00BB4H 00D60H 001ADH _DNET_TEXT             CODE
 00D62H 00F59H 001F8H _TEXT                  CODE
 00F60H 0146AH 0050BH COMDAT_SEG1            CODE
 0146CH 016F9H 0028EH _DATA                  DATA
 016FAH 01712H 00019H STRINGSEGMENT          DATA
 01714H 01714H 00000H XIFB                   DATA
 01714H 01714H 00000H XIF                    DATA
 01714H 01714H 00000H XIFE                   DATA
 01714H 0171BH 00008H CONST                  CONST
 0171CH 017B3H 00098H _BSS                   BSS

 Origin   Group
 0146:0   DGROUP

  Address         Publics by Name

 00F6:04F8       ??_C@_03HJFF@?$CD69?$AA@
 00F6:04EC       ??_C@_0M@OCLK@?40123456789?$AA@
 00F6:04FC       ??_C@_0P@MCIL@ncacn_dnet_nsp?$AA@
 00F6:011C       CLIENTCLOSE
 00F6:0000       CLIENTOPEN
 00F6:0178       CLIENTREAD
 00F6:02B4       CLIENTTOWERCONSTRUCT
 00F6:03CE       CLIENTTOWEREXPLODE
 00F6:0138       CLIENTWRITE
 0000:019A       EXPORTTIME
 0000:009F       I_DOSATEXIT
 0000:01AC       I_NSGETMEMORYALLOCATOR
 0000:00F8       I_RPCALLOCATE
 0000:00FE       I_RPCFREE
 0000:0104       I_RPCFREEBUFFER
 0000:010A       I_RPCGETBUFFER
 0000:0116       I_RPCNSBINDINGSETENTRYNAME
 0000:01A0       I_RPCREGISTEREDBUFFERALLOCATE
 0000:01A6       I_RPCREGISTEREDBUFFERFREE
 0000:0110       I_RPCSENDRECEIVE
 0000:0152       I_RPCTRANSCLIENTMAXFRAG
 0000:00B8       I_RPCTRANSCLIENTREALLOCBUFFER
 0000:013A       NDRCCONTEXTBINDING
 0000:0140       NDRCCONTEXTMARSHALL
 0000:0146       NDRCCONTEXTUNMARSHALL
 0000:015E       NDRCLIENTCONTEXTMARSHALL
 0000:018E       NDRCLIENTCONTEXTUNMARSHALL
 0000:0182       NDRCLIENTINITIALIZE
 0000:0188       NDRCLIENTINITIALIZENEW
 0000:017C       NDRCONVERT
 0000:016A       NDRFREEBUFFER
 0000:0170       NDRGETBUFFER
 0000:0176       NDRPOINTERBUFFERSIZE
 0000:0164       NDRPOINTERMARSHALL
 0000:0158       NDRPOINTERUNMARSHALL
 0000:0194       NDRSENDRECEIVE
 0000:01B8       NDRSIMPLESTRUCTBUFFERSIZE
 0000:01B2       NDRSIMPLESTRUCTMARSHALL
 0000:00CC       RPCBINDINGCOPY
 0000:00EC       RPCBINDINGFREE
 0000:00E0       RPCBINDINGFROMSTRINGBINDING
 0000:00DB       RPCBINDINGTOSTRINGBINDING
 0000:00E6       RPCBINDINGVECTORFREE
 0000:00BD       RPCGETEXCEPTIONHANDLER
 0000:00C7       RPCLEAVEEXCEPTION
 0000:0128       RPCREGCLOSEKEY
 0000:0122       RPCREGCREATEKEY
 0000:011C       RPCREGOPENKEY
 0000:0134       RPCREGQUERYVALUE
 0000:012E       RPCREGSETVALUE
 0000:00C2       RPCSETEXCEPTIONHANDLER
 0000:014C       RPCSSDESTROYCLIENTCONTEXT
 0000:00D1       RPCSTRINGBINDINGCOMPOSE
 0000:00D6       RPCSTRINGBINDINGPARSE
 0000:00F2       RPCSTRINGFREE
 00F6:04DC       TRANSPORTLOAD
 00D6:00E6       _atoi
 00BB:0004       _bcmp
 00BB:002D       _bcopy
 00BB:0052       _bzero
 0000:0063       _CallExport
 007E:000E       _connect
 00BB:0074       _decnet
 001B:000E       _dnet_addr
 0146:0134       _dnet_copyright
 002A:000C       _dnet_path
 0146:0176       _dnet_version
 0146:0132       _dnp_status
 0000:0000       _DOSDLLInit
 0146:02BC       _edata
 0146:0354       _end
 0048:005C       _endnodeent
 0146:003C       _errno
 0000:0046       _ExportInit
 0000:00A4       _GETENV
 0000:0081       _GetExportTableVersion
 003A:000E       _getnodebyaddr
 0041:0000       _getnodebyname
 0048:00FC       _getnodedb
 0048:007E       _getnodeent
 0000:00B3       _GETPROCADDRR
 002A:00F0       _get_current_volume
 005C:0000       _hclose
 005F:0004       _hopen
 0069:0002       _hread
 006F:0006       _hseek
 00BB:00EF       _install_check
 0000:00A9       _LOADMODR
 00B9:0006       _lohi
 00B9:0012       _lsw
 00D6:019C       _memcpy
 00BB:0116       _msdos
 00B9:001A       _msw
 0084:0002       _recv
 0078:000E       _sclose
 0095:0004       _select
 00A4:0000       _send
 0048:000E       _setnodeent
 00B3:000C       _socket
 0084:0062       _sread
 00D6:0012       _strcat
 00D6:00A2       _strcmp
 00D6:0066       _strcpy
 00D6:0140       _strcspn
 00D6:00CC       _strlen
 00A4:0054       _swrite
 0146:0048       _theTable
 0146:000C       _TransInfo
 0000:00AE       _UNLOADMODR
 0084:00A0       _xrecv
 00A4:0092       _xsend
 0000:0000  Abs  __ACRTUSED
 0000:0000  Abs  __ADBUSED
 0000:1000  Abs  __AHINCR
 0000:000C  Abs  __AHSHIFT
 00D6:00EA       __catox
 0146:0198       __ctype
 0146:0198       __ctype_
 0146:02BC       __edata
 0146:0354       __end
 0146:0046       __rpc_hostDS

  Address         Publics by Value

 0000:0000  Abs  __ACRTUSED
 0000:0000  Abs  __ADBUSED
 0000:0000       _DOSDLLInit
 0000:000C  Abs  __AHSHIFT
 0000:0046       _ExportInit
 0000:0063       _CallExport
 0000:0081       _GetExportTableVersion
 0000:009F       I_DOSATEXIT
 0000:00A4       _GETENV
 0000:00A9       _LOADMODR
 0000:00AE       _UNLOADMODR
 0000:00B3       _GETPROCADDRR
 0000:00B8       I_RPCTRANSCLIENTREALLOCBUFFER
 0000:00BD       RPCGETEXCEPTIONHANDLER
 0000:00C2       RPCSETEXCEPTIONHANDLER
 0000:00C7       RPCLEAVEEXCEPTION
 0000:00CC       RPCBINDINGCOPY
 0000:00D1       RPCSTRINGBINDINGCOMPOSE
 0000:00D6       RPCSTRINGBINDINGPARSE
 0000:00DB       RPCBINDINGTOSTRINGBINDING
 0000:00E0       RPCBINDINGFROMSTRINGBINDING
 0000:00E6       RPCBINDINGVECTORFREE
 0000:00EC       RPCBINDINGFREE
 0000:00F2       RPCSTRINGFREE
 0000:00F8       I_RPCALLOCATE
 0000:00FE       I_RPCFREE
 0000:0104       I_RPCFREEBUFFER
 0000:010A       I_RPCGETBUFFER
 0000:0110       I_RPCSENDRECEIVE
 0000:0116       I_RPCNSBINDINGSETENTRYNAME
 0000:011C       RPCREGOPENKEY
 0000:0122       RPCREGCREATEKEY
 0000:0128       RPCREGCLOSEKEY
 0000:012E       RPCREGSETVALUE
 0000:0134       RPCREGQUERYVALUE
 0000:013A       NDRCCONTEXTBINDING
 0000:0140       NDRCCONTEXTMARSHALL
 0000:0146       NDRCCONTEXTUNMARSHALL
 0000:014C       RPCSSDESTROYCLIENTCONTEXT
 0000:0152       I_RPCTRANSCLIENTMAXFRAG
 0000:0158       NDRPOINTERUNMARSHALL
 0000:015E       NDRCLIENTCONTEXTMARSHALL
 0000:0164       NDRPOINTERMARSHALL
 0000:016A       NDRFREEBUFFER
 0000:0170       NDRGETBUFFER
 0000:0176       NDRPOINTERBUFFERSIZE
 0000:017C       NDRCONVERT
 0000:0182       NDRCLIENTINITIALIZE
 0000:0188       NDRCLIENTINITIALIZENEW
 0000:018E       NDRCLIENTCONTEXTUNMARSHALL
 0000:0194       NDRSENDRECEIVE
 0000:019A       EXPORTTIME
 0000:01A0       I_RPCREGISTEREDBUFFERALLOCATE
 0000:01A6       I_RPCREGISTEREDBUFFERFREE
 0000:01AC       I_NSGETMEMORYALLOCATOR
 0000:01B2       NDRSIMPLESTRUCTMARSHALL
 0000:01B8       NDRSIMPLESTRUCTBUFFERSIZE
 001B:000E       _dnet_addr
 002A:000C       _dnet_path
 002A:00F0       _get_current_volume
 003A:000E       _getnodebyaddr
 0041:0000       _getnodebyname
 0048:000E       _setnodeent
 0048:005C       _endnodeent
 0048:007E       _getnodeent
 0048:00FC       _getnodedb
 005C:0000       _hclose
 005F:0004       _hopen
 0069:0002       _hread
 006F:0006       _hseek
 0078:000E       _sclose
 007E:000E       _connect
 0084:0002       _recv
 0084:0062       _sread
 0084:00A0       _xrecv
 0095:0004       _select
 00A4:0000       _send
 00A4:0054       _swrite
 00A4:0092       _xsend
 00B3:000C       _socket
 00B9:0006       _lohi
 00B9:0012       _lsw
 00B9:001A       _msw
 00BB:0004       _bcmp
 00BB:002D       _bcopy
 00BB:0052       _bzero
 00BB:0074       _decnet
 00BB:00EF       _install_check
 00BB:0116       _msdos
 00D6:0012       _strcat
 00D6:0066       _strcpy
 00D6:00A2       _strcmp
 00D6:00CC       _strlen
 00D6:00E6       _atoi
 00D6:00EA       __catox
 00D6:0140       _strcspn
 00D6:019C       _memcpy
 00F6:0000       CLIENTOPEN
 0000:1000  Abs  __AHINCR
 00F6:011C       CLIENTCLOSE
 00F6:0138       CLIENTWRITE
 00F6:0178       CLIENTREAD
 00F6:02B4       CLIENTTOWERCONSTRUCT
 00F6:03CE       CLIENTTOWEREXPLODE
 00F6:04DC       TRANSPORTLOAD
 00F6:04EC       ??_C@_0M@OCLK@?40123456789?$AA@
 00F6:04F8       ??_C@_03HJFF@?$CD69?$AA@
 00F6:04FC       ??_C@_0P@MCIL@ncacn_dnet_nsp?$AA@
 0146:000C       _TransInfo
 0146:003C       _errno
 0146:0046       __rpc_hostDS
 0146:0048       _theTable
 0146:0132       _dnp_status
 0146:0134       _dnet_copyright
 0146:0176       _dnet_version
 0146:0198       __ctype
 0146:0198       __ctype_
 0146:02BC       _edata
 0146:02BC       __edata
 0146:0354       _end
 0146:0354       __end

Program entry point at 0000:0000
